:100000000208F402030A75E05AF022020347750E53
:020010000222CA
:07001300020384750F0222B5
:07001B000203C1751002226F
:070023000205007511022225
:0B002B0002023EE4782DF22202053DA7
:03003B0002F110BF
:0300430002057A39
:03004B000205B7F4
:0300530002F100B7
:03005B000205F4A7
:0300630002063161
:03006B0002066E1C
:100073000202AAC0E0C0F0C083C082C0D074A575DC
:10008300E05A7582627583F078A5795A7AA57B5A0E
:100093007CA57D5A7EA57F5A18191A1B1C1D1E1F8D
:1000A30008090A0B0C0D0E0F25E028292A2B2C2DED
:1000B3002E2FF0A374FFF804F914FA04FB04FC04D4
:1000C300FD04FE14FF38393A3B3C3D3E3F58595A34
:1000D3005B5C5D5E5F540134A5345AF4F0A394A5D0
:1000E30098999A9B9C9D9E9FC8C9CACBCCCDCECFD5
:1000F300641068696A6B6C6D6E6F44014C4D4E4FB2
:10010300F0A3F074FF210BF0B42C01F0BB0801F055
:10011300BD0001F0BE0801F0BF0801F0D801F08076
:1001230001F020E001F020E101F020E201F020E302
:1001330001F020E401F020E501F020E601F020E7E2
:1001430001F0D34001F075E00110E001F075E0002B
:1001530030E00475E0A5F030E10475E0A5F030E28D
:100163000475E0A5F030E30475E0A5F030E4047510
:10017300E0A5F030E50475E0A5F030E60475E0A5F0
:10018300F030E70475E0A5F0C3500475E0A5F07402
:10019300002401700475E0A5F09401600475E0A5E6
:1001A300F01207031200060201B175E0A5F0C08347
:1001B300C0829001BC74007304D082D083A3F07416
:1001C30001F82606160876FF08760008F6C62829E1
:1001D3002A2B2CC423C3330300E675F002A413F0C7
:1001E300A3A2E6E5D0F58CE58C757FA5A67F8C7F71
:1001F3008D7F8E7F8F7FF57F457F657F957FD2795A
:100203009279A279F0D0D0D082D083D0F0D0E0E43C
:10021300782EF2FF1206F8E0FE782EE22EF2120696
:10022300F8E4F00FBF08ED782EE2643590F06160DA
:1002330005E04402F022E054FDF022C0E0C0F0C02B
:1002430083C082C0D075D000C000C001C002C0030B
:10025300C004C005C006C007E5B954207029538FF8
:10026300FEC2C77420F5B9120FEC1212DF121E84FE
:10027300121800121A19121E32121DD9120D4B1226
:100283000EDAE4F5B980057F20120BC3D007D00640
:10029300D005D004D003D002D001D000D0D0D0827A
:1002A300D083D0F0D0E032C0E0C0F0C083C082C0C1
:1002B300D075D000C000C001C002C003C004C00597
:1002C300C006C007538FFE75BF00E5BC540164012F
:1002D3007005121FB58015E5BC540264026008E581
:1002E300BC5410641070057F30120BC3D007D006C6
:1002F300D005D004D003D002D001D000D0D0D0821A
:10030300D083D0F0D0E032C0E0C0F0C083C082C060
:10031300D075D000C000C001C002C003C004C00536
:10032300C006C0077F90120BC3D007D006D005D0FC
:1003330004D003D002D001D000D0D0D082D083D05B
:10034300F0D0E032C0E0C0F0C083C082C0D075D02E
:1003530000C000C001C002C003C004C005C006C085
:10036300077F90120BC3D007D006D005D004D0036B
:10037300D002D001D000D0D0D082D083D0F0D0E052
:1003830032C0E0C0F0C083C082C0D075D000C000CE
:10039300C001C002C003C004C005C006C0077F90EF
:1003A300120BC3D007D006D005D004D003D002D09F
:1003B30001D000D0D0D082D083D0F0D0E032C0E0E2
:1003C300C0F0C083C082C0D075D000C000C001C0DF
:1003D30002C003C004C005C006C0077F90120BC350
:1003E300D007D006D005D004D003D002D001D0006E
:0B03F300D0D0D082D083D0F0D0E03218
:10040000005EBCE2613FDD83C29C7E20A3FD1F41F4
:100410009DC3217FFCA2401E5F01E3BD3E6082DCE4
:10042000237D9FC1421CFEA0E1BF5D0380DE3C62D4
:10043000BEE0025CDF81633D7C22C09E1D43A1FFC4
:100440004618FAA427799BC584DA3866E5BB5907B4
:10045000DB856739BAE406581947A5FB7826C49AA4
:10046000653BD987045AB8E6A7F91B45C6987A2494
:10047000F8A6441A99C7257B3A6486D85B05E7B984
:100480008CD2306EEDB3510F4E10F2AC2F7193CD74
:10049000114FADF3702ECC92D38D6F31B2EC0E5064
:1004A000AFF1134DCE90722C6D33D18F0C52B0EE54
:1004B000326C8ED0530DEFB1F0AE4C1291CF2D7344
:1004C000CA947628ABF517490856B4EA6937D58B34
:1004D0005709EBB536688AD495CB2977F4AA481624
:1004E000E9B7550B88D6346A2B7597C94A14F6A814
:1004F000742AC896154BA9F7B6E80A54D7896B3504
:10050000C0E0C0F0C083C082C0D075D000C000C0C1
:1005100001C002C003C004C005C006C0077F90121E
:100520000BC3D007D006D005D004D003D002D00131
:10053000D000D0D0D082D083D0F0D0E032C0E0C0A4
:10054000F0C083C082C0D075D000C000C001C0021E
:10055000C003C004C005C006C0077F90120BC3D003
:1005600007D006D005D004D003D002D001D000D0EF
:10057000D0D082D083D0F0D0E032C0E0C0F0C083D1
:10058000C082C0D075D000C000C001C002C003C08E
:1005900004C005C006C0077F90120BC3D007D00669
:1005A000D005D004D003D002D001D000D0D0D0826A
:1005B000D083D0F0D0E032C0E0C0F0C083C082C0B1
:1005C000D075D000C000C001C002C003C004C00587
:1005D000C006C0077F90120BC3D007D006D005D04D
:1005E00004D003D002D001D000D0D0D082D083D0AC
:1005F000F0D0E032C0E0C0F0C083C082C0D075D07F
:1006000000C000C001C002C003C004C005C006C0D5
:10061000077F90120BC3D007D006D005D004D003BB
:10062000D002D001D000D0D0D082D083D0F0D0E0A2
:1006300032C0E0C0F0C083C082C0D075D000C0001E
:10064000C001C002C003C004C005C006C0077F903F
:10065000120BC3D007D006D005D004D003D002D0EF
:1006600001D000D0D0D082D083D0F0D0E032C0E032
:10067000C0F0C083C082C0D075D000C000C001C02F
:1006800002C003C004C005C006C0077F90120BC3A0
:10069000D007D006D005D004D003D002D001D000BE
:1006A000D0D0D082D083D0F0D0E032538FFE75C04E
:1006B0000475C11675C23075C3F875C4FF75C5FFE2
:1006C000D2AD75BB13E4F5B8F5B975F812F5F9D2EA
:1006D000AF22120A0C1212B8121E9B121F28121EF1
:1006E0006E1217CC121F49121EBB12002E1209C126
:1006F0001206AB12104D80FB74622FF582E434F0C9
:10070000F5832275E0A5A3F0A322E709F608DFFA36
:100710008046E709F208DFFA803E88828C83E70989
:10072000F0A3DFFA8032E309F608DFFA8078E30904
:10073000F208DFFA807088828C83E309F0A3DFFA85
:10074000806489828A83E0A3F608DFFA8058898270
:100750008A83E0A3F208DFFA804C80D280FA80C658
:1007600080D4806980F28033801080A680EA809AED
:1007700080A880DA80E280CA803389828A83ECFA9A
:10078000E493A3C8C582C8CCC583CCF0A3C8C582F6
:10079000C8CCC583CCDFE9DEE7800D89828A83E49B
:1007A00093A3F608DFF9ECFAA9F0EDFB2289828A1F
:1007B00083ECFAE0A3C8C582C8CCC583CCF0A3C83B
:1007C000C582C8CCC583CCDFEADEE880DB89828ABB
:1007D00083E493A3F208DFF980CC88F0EF60010E88
:1007E0004E60C388F0ED2402B4040050B9F582EBEA
:1007F0002402B4040050AF232345822390075A7388
:10080000EF5BFFEE5AFEED59FDEC58FC22EB9FF535
:10081000F0EA9E42F0E99D42F0EC6480C864809862
:1008200045F022EB9FF5F0EA9E42F0E99D42F0E8A8
:100830009C45F022E8600FECC313FCED13FDEE13B2
:10084000FEEF13FFD8F122E6FC08E6FD08E6FE08FD
:10085000E6FF22E0FCA3E0FDA3E0FEA3E0FF22E42C
:1008600093FC740193FD740293FE740393FF22E4DE
:1008700093F8740193F9740293FA740393FB22ECD6
:10088000F0A3EDF0A3EEF0A3EFF022A8828583F0B1
:10089000D083D0821208A21208A21208A21208A2C3
:1008A000E473E493A3C583C5F0C583C8C582C8F0CB
:1008B000A3C583C5F0C583C8C582C822A42582F517
:1008C00082E5F03583F58322D083D082F8E49370FB
:1008D00012740193700DA3A393F8740193F58288A9
:1008E00083E4737402936860EFA3A3A380DF8A8319
:1008F0008982E47375BF0375B3F075BF0078007F1C
:1009000000E4F208DFFC7581AD0209470206D2E47B
:1009100093A3F8E493A34003F68001F208DFF48088
:1009200029E493A3F85407240CC8C333C4540F44D8
:1009300020C8834004F456800146F6DFE4800B01B2
:100940000204081020408090098CE47E019360BC72
:10095000A3FF543F30E509541FFEE493A360010E4A
:10096000CF54C025E060A840B8E493A3FAE493A371
:10097000F8E493A3C8C582C8CAC583CAF0A3C8C592
:1009800082C8CAC583CADFE9DEE780BEC105010CA3
:1009900000010D0000000000000A050069010101CE
:1009A0000101010101000000000000000000000042
:1009B0000000000000000000000000000000000037
:1009C00000E4F5B25380FC75B20343800375B201B5
:1009D0005386FCF5B243860353901C75B2034390D3
:1009E000E375B20153911CF5B24391E343A17875CD
:1009F000B20153A187F5B253B04375B20343B0BC03
:100A000075B20153B143F5B243B1BC22E4F5BF75F1
:100A1000BB1290F06AF090F061F012230C50069037
:100A2000F06A7420F090F07274FFF090F073740824
:100A3000F051CC500790F06AE04410F090F07274DE
:100A400007F0E490F073F043D00851CC920053D0FB
:100A5000F730000790F06AE04410F0122026902F43
:100A6000FFE4936F600790F06AE04440F012206664
:100A7000501C90F06AE04401F0E5BC5440600FE087
:100A80004402F053BCBFA3E5BDF0A3E5BCF01200E7
:100A90007612209A90F06DEFF0600790F06AE044D3
:100AA00008F0E4782CF290F06E74A0F0A3E4F090DB
:100AB000F07074A8F0A3E4F012194C90F061E070AB
:100AC0000690F06AE060047F3071C32275BF037541
:100AD000B3F1E4F5BFC2D190F072E0FFFE90F07385
:100AE000E06F6011C8EFC8E6C8EEC8F2C8EFC8E40E
:100AF000F61F1E80E8C8EFC8E6C8EEC8F2C8EFC807
:100B0000E4F690F072E06F600FC8EFC8E67004760C
:100B1000FF8002D2D10F80EAC8EFC8E6700476FFEA
:100B20008002D2D190F073E0FF90F072E06F60101D
:100B3000C8EFC8E6B4FF04E4F68002D2D10F80E922
:100B4000C8EFC8E6B4FF04E4F68002D2D190F07397
:100B5000E06F600FC8EFC8E6700476FF8002D2D164
:100B60001F80EAC8EFC8E6700476FF8002D2D190F9
:100B7000F072E0FF90F073E0FD6F6010C8EFC8E620
:100B8000B4FF04E4F68002D2D11F80E8C8EFC8E6C3
:100B9000B4FF04E4F68002D2D1CEEDCE90F072E044
:100BA0006E600CC8EEC8E2C8EFC8F60F0E80EDC844
:100BB000EEC8E2C8EFC8F675BF0375B3F0E4F5BF41
:100BC000A2D122122488EF440B121FD17891E6445F
:100BD00002F6F4782BF6801E7887762D742DF47843
:100BE00021F67892768A748AF4782CF67891E64425
:100BF00001F6F4782BF61225508FB0E58054FBFFF8
:100C000090A6E4E49342078F802212262BFE8F33B6
:100C10007890E6FF782A6652068F367891E6FF785C
:100C20002B6652068F35853334EEF4600281F6E58B
:100C30003311C80CE60F0C891E0CC32D0C713C0C33
:100C400052690C5E780C9C960CB6A50CA9B40000F9
:100C50000CEEE535540A640A7002A10480177893FB
:100C6000E6B494028064E5366002A10475343CA1C8
:100C700004E5366005753478A1047893E6648A60EB
:100C800002A104F675341E807BE536600280087888
:100C900093E66485706EF67534968068E51270058B
:100CA0007534B4805F1512805BE51270057534A54C
:100CB00080521512804EE512700575342D80451551
:100CC0001280417893E6FFB49407E4F675344B80C4
:100CD00033EF64C9702EE535702AE53670267893B7
:100CE000F675340F801E12245A1224F380FE12244B
:100CF000881225BE800C1225BE1225B312248885C9
:100D0000333471F6E53465336040E53424B5601F53
:100D100024A6601224F16009241E702290A6D480BB
:100D20000890A6D5800390A6D6E493F512800F1202
:100D300025EEA634D1DA1210B512109580FB1225DB
:100D4000EEE6B53303A6342271D82205137889E67E
:100D5000FF782366FE122506400C15327889A632EC
:100D6000E532F47823F690A6CE12247B5004440298
:100D7000800254FDF6F4782AF6788AE6FF78241289
:100D80002503400C1532788AA632E532F47824F631
:100D900090A6CF12247B50044404800254FBF6F446
:100DA000782AF6788BE6FF7825122503400C153259
:100DB000788BA632E532F47825F690A6D012247B03
:100DC00050044408800254F7F6F4782AF6788CE64A
:100DD000FF7826122503400C1532788CA632E532B6
:100DE000F47826F690A6D112247B50044410800299
:100DF00054EFF6F4782AF67888E6FF782212264334
:100E00007C005403FD7013E532D39401400C15327D
:100E10007888A632E532F47822F612247F50044412
:100E200001800254FEF6F4782AF6788DE6FF7827E2
:100E30006652068F32ED4C7013E532D39401400CAC
:100E40001532788DA632E532F47827F690A6D212C4
:100E5000247B50044420800254DFF6F4782AF6788C
:100E60008EE6FF782812264354037013E532D3949C
:100E700001400C1532788EA632E532F47828F690CF
:100E8000A6D312247B50044440800254BFF6F47869
:100E90002AF6788FE6FF78296652068F3212247F71
:100EA000500444808002547FF6F4782AF6BEFF1680
:100EB0007893E6B4A914788F76807480F47829F654
:100EC000E47893F680047F80D1CC810A122488EFE5
:100ED000440A121FD11225B361F6538FFEE4F5B216
:100EE00012262B8F37F47022E537540FFFE5B054EC
:100EF000FCFEEF90A6E79342068EB0E58054FBFE21
:100F0000EF90A6D79342068E80227F80F11061F683
:100F1000122488EF440D121FD17891E64404F6F4B0
:100F2000782BF661F6122488121FCE61F612251F67
:100F30008C3A12260012250E1224DB1225DC122513
:100F40000E1224A3E493601D24FE600D047026128B
:100F50002432C3110D601A8014122432C3110D40C3
:100F600002800A800C122432D3110D50047F30808D
:100F700031E4FF80047F9080AC8F477828E6F4FF4F
:100F8000788EE6FE6F701990A6CC12241F4006766C
:100F90008074808006788EEF26F6E6F47828F622B4
:100FA00061D87828E6F4FE788EE6FD6E701C90A677
:100FB000CD93FEC39D4006760174018006C3788EF2
:100FC000E69EF6F47828F6021FCE61D8122488EF48
:100FD0004406121FD161F6122488EF440E121FD16D
:100FE0007891E64408F6F4782BF661F690F061E02B
:0D0FF000700690F06AE060047F3071C3224B
:10100000E5B0544060FA43AB8053B5FD53B5FB786F
:1010100024E2F5ACE5B5540260FA53B5FD7825E25B
:10102000F5ACE5B5540460FA53B5FB7823E5ADF2B1
:10103000E5B5540260FA53B5FD7824E2F5ACE5B0AD
:10104000544060FA7822E5ADF253AB7F22E4F5BF5D
:1010500053BBBF1200767F1051649200782CE204DB
:10106000F2E2B48014E4F290F06E74A0F0A3E4F025
:1010700090F07074A8F0A3E4F030000790F06AE0FC
:101080004404F090F061E0700690F06AE060057F43
:1010900030120BC322E5B0544060FA1225E5E27825
:1010A0002A122526EFF21225E5E27828122526EFEE
:1010B000F2312480E0C2AFE4F5FEF5FF539DFB78EA
:1010C00024F208F2C205D20430045811007822122A
:1010D000263B64027004E53764AB600A087412F2C0
:1010E000087434F280097824E537F208E538F21103
:1010F0000078247456F2087478F27822E2F5390800
:10110000E2F53AE538B402C0E537B4ABBBE53AB432
:10111000B6B6E539B4A5B1C2040874ABF208744B95
:10112000F280A522782A12263B7829E2540FFBE2AE
:101130005480AF03AD38AC37700241328C398D3AF0
:10114000EF24FE604514601314602F24FE604214E7
:101150006046147046AF3AAE398068E4B53A12E59D
:1011600039B4A00D31A35006782474028007E480BE
:101170002C78247403F208E4F2227828E2FFE5399F
:1011800054F1853A82F583EFF0227828E2A83AF606
:1011900022AA39A93A0208EE02200074AA7824F2A1
:1011A00008F222E4F5BFF5BC75BF0143E901F5BFC4
:1011B000781B76FF08760308F608F608F612DFF9C2
:1011C000022633C3EE94A050028009D3EF94FFEEC1
:1011D00094AF400678247404803D2005127826EEF2
:1011E000F208EFF2D20578217460F2E418F2227866
:1011F00028E2FF7820E2FE08E22EF8A6077820E237
:1012000004F2E2C3942040167826E2FE08E2FF5181
:101210001F500978247408F208E4F222C20522E47F
:10122000F5BFF5BC781876608F828E8312DFF602E8
:1012300026338D828C83EF24FE601524FE60082403
:10124000FC7019E493800EE58354F1F583E080058A
:10125000AF82A807E67825F2E418F22274AA78246F
:10126000F208F22290F06EE0F530A3E0F531A3E051
:10127000FCA3E0FDC201853182853083E493F4FE56
:101280008D828C83E4936E60047E0180027E00EE8A
:101290006004D201800F0531E531700205300DBDCB
:1012A00000010CDFD190F06EE530F0A3E531F0A342
:1012B000ECF0A3EDF0A201227F2CE4C39F500F1F9E
:1012C000EF90099593FE74802FF8A60680EC538F5B
:1012D000FE75BF0178AC762808A6B3E4F5BF22E519
:1012E0000C650D602AE50D540FFE25E02401F8E29F
:1012F000547FFFEE25E02400F8E2FD7110C3E50CF9
:10130000950DD39408400443170122050D80D02287
:10131000EFC39404400BEFD394124068EF942C5029
:1013200063EF24E9600F24FE600E24FE600D2406A6
:10133000700C02000E02001602001E0200267480CD
:101340002FF8A605EF1208C8136A00137914137B4F
:1013500016137E1813811A13711C13741D13771E34
:10136000136C24136F2900001384A16702183C80BA
:1013700014021D25021CFEE128E1F2021F9D021F3E
:10138000A5121FAD22E4F532F533F537F536F53504
:10139000F534F538F539122443E078A9666007057D
:1013A00033E533B408F0E533C3940840057F1002F9
:1013B0000FA278A9E6F53212244374FFF075F00607
:1013C000E53290A1601208BCE493B40700400281AA
:1013D0005E9013D725E073812D811161F0815681D4
:1013E00041813661E512240F1224D81225D4A1CEF2
:1013F00078A51208478F378E368D358C3412240F1E
:101400001224D8853242AF37AE36AD35AC34020F38
:101410002D78A7E6F53808E6F53912240F1208539F
:10142000AD07AC06AE38AF39AB3202189412240FB8
:1014300012257702190012240F1224D81225D48005
:101440002212240F120853AD07AC0678A7E6FE0857
:10145000E6FFAB32A10A12240F122577804F7F904E
:10146000020F251224A3E493602724FE6012047067
:10147000371223E3122493FCC31208236025801E35
:101480001223E3122493FCD31208235002800F800E
:10149000121223E3122493FCC312082340057F3069
:1014A000020FA2E4FF020F797F90020F258F3AA965
:1014B0000575F006EB1224B0E493602E24FE60154F
:1014C00004704275F006EB122406E53A5FFEEF5910
:1014D0006E602D802675F006EB122406E53A5FFE5D
:1014E000EF59C39E40028013801675F006EB12245C
:1014F00006E53A5FFEEF59D39E50057F30020FA2FA
:10150000E4FF020F797F90020F25122611A90375BF
:10151000F006E91224B0E493602E24FE60160470F5
:101520004175F006E91224061224C86D7002EE6CB3
:10153000602B802475F006E91224061224C8C39D8E
:10154000EE9C40028012801575F006E91224061206
:1015500024C8D39DEE9C50057F30020FA2E4FF0209
:101560000F797F90020F2575F005E51590A0011207
:1015700008BCE493788066FF75F005E51590A0023D
:1015800012254675F005E51590A00312254675F065
:1015900005E51590A004122546EF702A90A140930E
:1015A000FFE514C39F401B051590A142E493FFE59E
:1015B000159F4003E4F515122536F6E4FF1219C510
:1015C00080087F2080027F30F19EE4F514221225EE
:1015D0001F8C3AE4F543F544F545F54612255DE4E4
:1015E000FBFA7980787FC31208237002E123122569
:1015F0006AFCE4787FC31208237002E11F12256A97
:10160000FC78171208348F44E412255D781712080D
:10161000348F43E4FFFEFDE53A1226098F46E4FFCE
:10162000FEFDE53E1226098F45E544700912259B13
:10163000EF4480FF800712259BED4480FDE41225D6
:101640001FF53AE543700912258FEF4480FF8007AC
:1016500012258FED4480FDE41225F7E544C3954340
:1016600050141225DCC3E5439544F9F812083412EE
:10167000251F8C3A8016E544D39543400F1226006F
:10168000E5449543F9F81208341224DB122401EFE3
:10169000553DFFEE553CFEED553BFDEC553A122510
:1016A0001FF53A1224011224931225F71224ABE4F9
:1016B00093603224FE7064E5456546701DE545B4CF
:1016C000800B122432D31208234046804912243260
:1016D000C31208235002803E8037E545C39546502B
:1016E00002802E8031E5456546701FE545B4800DCA
:1016F000122432C31208235002801B801412243299
:10170000D31208234002800E8007E545D39546405A
:10171000057F30020FA2E4FF020F797F9080067FE1
:101720008080027F80020F25789FE630E703122039
:101730000012200653B0BF789FE6FDD3940B4005FE
:101740007F80020FD7789EE6FFC2AFE4F5BF43BBB0
:101750000175BF01782DE5BAF243B50143B50843E1
:10176000B50443B50275BF0143B70843B70443B698
:1017700010ED540F42BA43B41012245D8FBC43BB2A
:10178000011224F9438F0143BB02538FFE75BF0141
:1017900075BB9B43B40875BBAB538FFE80FE7822AC
:1017A000E6F4FE7888E6FD6E701F90A6C193FEC336
:1017B0009D4006760174018006C37888E69EF6F4A3
:1017C0007822F6EF4401021FD1020BD8E4FB90F01F
:1017D0002FF0A374FFF0EB12244574FFF01224E401
:1017E000E4F0EB12241112088B000000000BBB0880
:0A17F000E522E47895F6750E01225B
:10180000E4FC1225C96FAB06F4702CEC122445E001
:10181000C394805014EC1224E5E0B5030C7F201231
:101820000FA2EC12244574FFF00CBC08DE0B90F004
:101830002FEBF0F4A3F0227F80020F25E4FB1225AA
:10184000C96FAA06F4704890A46193FF78A4E6C318
:101850009F503AEBC39408500BEB122445E0F46020
:10186000030B80EFEBC39408502578A0120847EBD8
:1018700012241112087F90A460E4932AFF1224E43A
:10188000EFF078A4E6FFEB122445EFF02280007F12
:1018900080020F25122611E4FFFE75F006EB1224DC
:1018A000061224D0FF8E3CF53D75F006EB1224069F
:1018B000E53A5EFEE53B5F8E3AF53B75F006EB12CE
:1018C00024B0E493602224FE601104702EE53D658F
:1018D0003B7004E53C653A601D8016C31225A76481
:1018E00080984002800B800ED31225A76480985008
:1018F000057F30020FA2E4FF020F797F90020F25CF
:10190000AA05A907E4FF75F006EB122406AE07EA64
:101910005EFAE95EF975F006EB1224B0E493601705
:1019200024FE6009047020EA6960178010C3122643
:101930001A40028008800BD312261A50057F30020D
:101940000FA2E4FF020F797F90020F2578887601BD
:101950007401F47822F6788976017401F47823F61C
:10196000788A76017401F47824F6788B7601740114
:10197000F47825F6788C76017401F47826F6788D63
:1019800076017401F47827F6788E76017401F47884
:1019900028F6788F76017401F47829F6E4F1D1788D
:1019A00090767F747FF4782AF6E47891F6F4782BB9
:1019B000F6E47893F6788776697469F47821F6E42A
:1019C000F513F512228F327822E6F4FF7888E6FECE
:1019D0006F701990A6C012241F4006768074808014
:1019E000067888EF26F6E6F47822F622020BD88FE6
:1019F000347823E6F4FF7889E6FE6F701990A6C26A
:101A000012241F40067680748080067889EF26F6BF
:101A1000E6F47823F622020BD8E4FBFAF532F5332C
:101A200075D106F5D243CD40F5D1F1EB60FC75D10F
:101A300002E50E6021B401097895F1D918E6FB8022
:101A400010E5CAF1DAABCBE50EB40205750E0380E2
:101A500015E4F50E8010E5CA54C07895F618A6CBAB
:101A6000E5CAF1DAABCB1224B690A6A0F1E1500D95
:101A700090A6A2F1E14006E4FF31EF80047F3091AF
:101A80004D75D10675D201F1F2F1EB60FC75D10212
:101A9000E50F6021B401097897F1D918E6FB8010B1
:101AA000E5CCF1DAABCDE50FB40205750F03801577
:101AB000E4F50F8010E5CC54C07897F618A6CDE574
:101AC000CCF1DAABCD1224B690A6A4F1E1500D9082
:101AD000A6A6F1E14006E4FF71CF80047F30917A41
:101AE00075D10675D202F1F2F1EB60FC75D102E519
:101AF000106021B401097899F1D918E6FB8010E54E
:101B0000CEF1DAABCFE510B402057510038015E411
:101B1000F5108010E5CE54C07899F618A6CFE5CE22
:101B2000F1DAABCF1224B690A6A8F1E1500D90A641
:101B3000AAF1E14006E4FF71F980047F3091A775B6
:101B4000D10675D207F1F2F1EB60FC75D102E51117
:101B50006021B40109789BF1D918E6FB8010E5D229
:101B6000F1DAABD3E511B402057511038015E4F584
:101B7000118010E5D254C0789BF618A6D3E5D2F1B7
:101B8000DAABD3EB75F004A4FFAD021224BE90A62D
:101B9000ACF1E1500B90A6AEF1E14004E4FF8123EB
:101BA0007F307826E6F4FE788CE6FD6E701E90A6F7
:101BB000C993FEC39D4006760174018006C3788CEC
:101BC000E69EF6F47826F6EF4405E1D1020BD88FB5
:101BD000347824E6F4FF788AE6FE6F701990A6C484
:101BE00012241F4006768074808006788AEF26F6DD
:101BF000E6F47824F622020BD88F347825E6F4FF39
:101C0000788BE6FE6F701990A6C612241F400676E8
:101C10008074808006788BEF26F6E6F47825F6222D
:101C2000020BD88F347826E6F4FF788CE6FE6F70CE
:101C30001990A6C812241F4006768074808006780A
:101C40008CEF26F6E6F47826F622020BD87823E607
:101C5000F4FE7889E6FD6E701E90A6C393FEC39DC8
:101C60004006760174018006C37889E69EF6F47812
:101C700023F6EF4402E1D1020BD87824E6F4FE7893
:101C80008AE6FD6E701E90A6C593FEC39D40067643
:101C90000174018006C3788AE69EF6F47824F6EF94
:101CA0004403E1D1020BD87825E6F4FE788BE6FDFB
:101CB0006E701E90A6C793FEC39D40067601740108
:101CC0008006C3788BE69EF6F47825F6EF4404E1AF
:101CD000D1020BD88F347827E6F4FF788DE6FE6FBB
:101CE000701990A6CA12241F400676807480800660
:101CF000788DEF26F6E6F47827F622020BD8789D49
:101D0000E6FBC204E4FAEA122453B5030576FF1297
:101D100026230AEAC3940850033004EA2004057F0E
:101D200080120FCC22C204E4FB789CE6FAE54865F9
:101D30004AFF854832E549654B5207854933EFF440
:101D4000706475F002E53290A4801208BCE4936AD6
:101D50007050EB122453F4703AA60275F002E5328B
:101D600090A4811208BCE4932533FFEB25E0244DB9
:101D7000F8A607E53204FF90A67EE493FEEFC39E2B
:101D800050088F48EFF4F54A8006E4F548754AFF9D
:101D90001226230BEBC3940850033004B520040B28
:101DA00080047F1080067F80120FCC227827E6F413
:101DB000FE788DE6FD6E701E90A6CB93FEC39D400F
:101DC00006760174018006C3788DE69EF6F47827C6
:101DD000F6EF4406E1D1020BD8E549654B8549325F
:101DE000F47023FCEC122453F4600EEC25E0244D37
:101DF000F8E6B532047F20B1AC0CBC08E7E532044C
:101E0000F549F4F54B227F80020FCC7829E6F4FEE9
:101E1000788FE6FD6E701804C39D4006760174014C
:101E20008004788F16E6F47829F6EF4408E1D102B1
:101E30000BD8AF17EF603630E0075317FE7F808076
:101E400022EF30E2155317FB7F40D10BE4122583BC
:101E500075AA0775A302439D0422EF30E1075317CB
:101E6000FD7F2080A6E4F5177F80120BC322E4F5E6
:101E700014F51590A140937885F6A3E49318F61213
:101E80002536F622051490A141E493FFE514D39F73
:101E90004008E4F5147F2012179E22538FFEE4F5CC
:101EA000B2122550E58054FBFE90A6E4E49342066E
:101EB00043B1038FB04386048E802275A30275FE62
:101EC0000775FF80539FFC439D0475A303539E3FFA
:101ED000D2EC75A30275B20175B04075B140E4F55E
:101EE000B275A90675B2024380205386DF75B2032E
:101EF000758020F5B243862012258375AA07D2E9A2
:101F0000F50CF50DF517C206750B55750A55C3741A
:101F1000A89400FF74F194F1FE7A2979007BFF7890
:101F2000007CF17D010207DAE4F548754AFFF549C6
:101F3000754BFFFFEF25E0244CF876FFEF25E024FA
:101F40004DF8E4F60FBF08EC22F155E4F50EF50F5D
:101F5000F510F51122E4F5D175CA8075CC51F5CD97
:101F6000F5CEF5CF75D101F5CA75CB0175CC0275EB
:101F7000D30375D10675CD01F5D275D10475CAC0EC
:101F800075CBC075CCC075CDC0F5CE75D105F5CB80
:101F9000F5CCF5CDF5CFF5D2F5D3F5D122E4789790
:101FA000F6750F0122E47899F675100122E4789B0A
:101FB000F67511012253BCFE75BF01782DE2F5BA0A
:101FC00075B60275B702E5B7540160FA80FEEF44BA
:101FD000077892F6F4782CF622E6C413135403FA29
:101FE000227401939533E493953222E5CB54016436
:091FF000012243CD40E4F5D122A9
:10200000915A91F380FE75A302539DFBE4F5FEF512
:10201000FF75B20175B0FFF5B275B14075B04043C0
:10202000B14043B040227530FF7F807E5F90040056
:1020300043A201E4F583F58243A201E493F9A3539B
:10204000A2FEF582E493FD6230DFED7F80DEE91FC2
:1020500043A201E493F9A353A2FEF582E493FD6247
:1020600030DFEDAF3022C2017F007EA87D007CA072
:102070008D828C83E493FB8F828E83E4936BF46078
:1020800004D20180120DBD00010C0FBF00010EE44F
:10209000B505DDECB4A8D9A20122E4F530FF90A18A
:1020A0004293FDD394404003753001EDC394085032
:1020B0000375300190A141E493FDD394644003750E
:1020C0003006EDC39401500375300690A140E493AF
:1020D000FDD39463400375300790A141E493C39D01
:1020E000500375300790A6C0E493D3944040037525
:1020F000301090A6C1E493D39440400375301790FC
:10210000A6D3E493707BFE90A461E493FDEEC39D9F
:10211000503575F006EEA42460F582E5F034A1F5A3
:1021200083E493D39406400375302575F006EEA43E
:102130002461F582E5F034A1F583E493D394024061
:10214000037530260E80C090A460E493FCD394FE07
:10215000400375300DECC39401500375300DEDD381
:102160009480400375300490A6CCE493D39440400F
:102170000375301690A6CDE493D394404003753098
:102180001D90A6D2E493704290A6CA93D394404087
:102190000375301590A6CBE493D39440400375307B
:1021A0001CE4FE90A67EE493FDEEC39D501C75F0EA
:1021B00002EEA42481F582E5F034A4F583E493C310
:1021C000940250037530270E80D990A6CEE4937008
:1021D0002BD390A6A2049394FFE493940340037539
:1021E000300E90A6C2E493D3944040037530119012
:1021F000A6C3E493D39440400375301890A6CFE46F
:1022000093702BD390A6A6049394FFE49394034079
:102210000375300E90A6C4E493D394404003753008
:102220001290A6C5E493D39440400375301990A64C
:10223000D0E493702BD390A6AA049394FFE49394D4
:1022400003400375300E90A6C6E493D39440400338
:1022500075301390A6C7E493D39440400375301AA9
:1022600090A6D1E493702BD390A6AE049394FFE490
:10227000939403400375300E90A6C8E493D3944022
:10228000400375301490A6C9E493D394404003757D
:10229000301BE4FEEE90A6E79354FC600375300C0F
:1022A000EE90A6D79354FB600375300C0EBE10E47D
:1022B00090A6D4E493D394FE400375300890A6D53D
:1022C000E493D394FE400375300990A6D6E493D3EB
:1022D00094FE400375300A90A6D3E493FF90A6D2F3
:1022E000E4934FFF90A6CFE493FD90A6CEE4934DE8
:1022F000420790A6D1E493FD90A6D0E4934D420707
:102300005307BFEF6003753024AF302290F061E0D7
:10231000F53090F06AE0F531C201C20275BF037575
:10232000B3F0E4F5BFF8F208E86005E4F20880F8DD
:10233000716C920175BF0375B3F1E4F5BF78FFF2DC
:1023400018E8F46005E4F21880F7716C920275BF2A
:102350000375B3F0E4F5BF90F061E530F090F06AFA
:10236000E531F0A20272019201A20122C203E4F857
:10237000E2700574FFF28002D20308E8600DE2709B
:102380000574FFF28002D2030880F0E2B4FF04E497
:10239000F28002D20308E8600DE2B4FF04E4F280A8
:1023A00002D2030880F078FFE2700574FFF2800229
:1023B000D20318E8F4600DE2700574FFF28002D2D7
:1023C000031880EFE2B4FF04E4F28002D20318E8BD
:1023D000F4600DE2B4FF04E4F28002D2031880EF4F
:1023E000A2032275F006E54290A1621208BC120811
:1023F0005FEF553DFBEE553CFAED553BF9EC553A98
:10240000F875F006E54290A1621208BC02085FE58B
:102410003375F006A42431F582E434F0F583229379
:10242000FFFDEE2DFDE433FCC3ED9480EC6480945D
:102430008022AF3DAE3CAD3BAC3AAB41AA40A93F98
:10244000A83E22E53375F006A42436F582E434F084
:10245000F5832225E0244CF8E622538FFE75BF0158
:1024600075BB9BE4F5BF438F0143BB04538FFE75DF
:10247000BF0175BBABF5BF438F0122E4934232E548
:1024800032C394407890E6227887762D742DF478C4
:1024900021F622EF5541FFEE5540FEED553FFDEC94
:1024A000553E228F3D8E3C8D3B8C3A75F006E542C1
:1024B00090A1610208BCEB75F004A4FFEAFDE5F011
:1024C000F532EF4DF533C322E53A5EFCE53B5FFDA7
:1024D000E53C5EFEE53D5F221208538F418E408D44
:1024E0003F8C3E22EB75F006A42435F582E434F0EF
:1024F000F5832275BCFF53BBFE43BB0243BB1053A5
:102500008FFE226652068F32E532D394012275F097
:1025100006E54290A1621208BC12086F0208008F03
:102520003D8E3C8D3B22CFF208EFF218E2FF08E22D
:102530007824CFF2082275F005E51590A000120866
:10254000BCE4937886221208BCE493086642072212
:10255000E5B054FCFF90A6F4E493420722FFFEE5A9
:102560003F5480FDE53E547FFC22E4FFFEE53B54F2
:1025700080FDE53A547F22120853AD0778A8E6FFA4
:10258000AB3222F5AF75AE0653AB7F75AB0422E5D7
:1025900041FFE540FEE53F547FFD22E53DFFE53C80
:1025A000FEE53B547FFD22E53D953BE53A6480F82E
:1025B000E53C227891E64401F6F4782BF6227892F5
:1025C000768A748AF4782CF62290F030E0FF90F04E
:1025D0002FE0FE2285324278A5020847AF3DAE3C8F
:1025E000AD3BAC3A221210007822E2FF0822E5341B
:1025F000F47821F67887228F418E408D3FF53E2278
:10260000AF41AE40AD3FAC3E225480FC781802088A
:10261000348E3A8F3B8C3C8D3D22E96480F8EA642D
:10262000809822E4FF121CD4D204227887E6FF7837
:10263000216622E4F5BF9204A20422E2F53708E203
:0B264000F538226652068F32E51322A7
:1029000043AB80850BAC539DFB75A30043A50432FC
:10291000C0E0C0D075D018E5B55404605785AD1639
:1029200053B5FB100607851609D206807685160872
:1029300075AB04E50930E71A85080B85090AE50C33
:10294000540F25E02400F8E508F208E509F2050C2B
:10295000800BE5092480F8E6F50B85090A75A302CA
:10296000439D04E5B05440703A750BAA750AAA431A
:102970001702802FE5B530E10653B5FD850AACE5B9
:10298000B530E01F53B5FE4317047F96E5B05440C1
:102990007002DFF875A302439D0453B5F9750BAAC5
:0929A000750AAAD0D0D0E0322261
:012FFF00AA27
:10A0000000F80DE97401B742A63B02EE1BFF6203A4
:10A01000A154B02D04728763FE053DC82CB10664BF
:10A020009175E8072BDE3AA708D520C459099A6F25
:10A030008B160AC336D24F0B8C799D000C5FAA4E4B
:10A04000D30D10E5019C0E49BC58C50F06F3178AC5
:10A050000000000000000000000000000000000000
:10A0600000000000000000000000000000000000F0
:10A0700000000000000000000000000000000000E0
:10A0800000000000000000000000000000000000D0
:10A0900000000000000000000000000000000000C0
:10A0A00000000000000000000000000000000000B0
:10A0B00000000000000000000000000000000000A0
:10A0C0000000000000000000000000000000000090
:10A0D0000000000000000000000000000000000080
:10A0E0000000000000000000000000000000000070
:10A0F0000000000000000000000000000000000060
:10A10000000000000000000000000000000000004F
:10A11000000000000000000000000000000000003F
:10A12000000000000000000000000000000000002F
:10A13000000000000000000000000000000000001F
:10A14000020B1000000000000000000000000000F2
:10A1500000000000000000000000000000000000FF
:10A160000002FFFFFFFF0401FFFFFF000200FF00EE
:10A1700000000602FFFF00000002FFFFFFFF0000DB
:10A18000FFFFFFFF0001FFFFFFFF0302FFFFFFFFD5
:10A190000300FFFFFFFF0301FFFFFFFF0402FFFFBC
:10A1A000FFFF0400FFFFFFFF0401FFFFFFFF0402AA
:10A1B000FFFFFF000400FFFFFF000401FFFFFF009F
:10A1C0000102FFFFFFFF0100FFFFFFFF0101FFFF93
:10A1D000FFFF0102FFFFFF000100FFFFFF00010181
:10A1E000FFFFFF000502FF0000000500FF00000068
:10A1F0000501FF0000000502FFFF00000500FFFF52
:10A2000000000501FFFF00000502FFFFFF00050041
:10A21000FFFFFF000501FFFFFF000502FFFFFF003A
:10A220000500FFFFFF000501FFFFFF000200FF0028
:10A2300000000200FF0000000201FF000000020019
:10A24000FFFF00000202FFFF00000201FFFF00000D
:10A250000200FFFFFF000202FFFFFF000201FFFFFD
:10A26000FF000200FFFF00000202FFFF00000201EA
:10A27000FFFF00000600FFFFFFFF0602FFFFFFFFDA
:10A280000602FFFFFFFF0000FFFFFFFF0000FFFFD0
:10A29000FFFF0000FFFFFFFF0000FFFFFFFF0000C8
:10A2A000FFFFFFFF0000FFFFFFFF0000FFFFFFFFBA
:10A2B0000000FFFFFFFF0000FFFFFFFF0000FFFFA8
:10A2C000FFFF0000FFFFFFFF0000FFFFFFFF000098
:10A2D000FFFFFFFF0000FFFFFFFF0000FFFFFFFF8A
:10A2E0000000FFFFFFFF0000FFFFFFFF0000FFFF78
:10A2F000FFFF0000FFFFFFFF0000FFFFFFFF000068
:10A30000FFFFFFFF0000FFFFFFFF0000FFFFFFFF59
:10A310000000FFFFFFFF0000FFFFFFFF0000FFFF47
:10A32000FFFF0000FFFFFFFF0000FFFFFFFF000037
:10A33000FFFFFFFF0000FFFFFFFF0000FFFFFFFF29
:10A340000000FFFFFFFF0000FFFFFFFF0000FFFF17
:10A35000FFFF0000FFFFFFFF0000FFFFFFFF000007
:10A3600000000000000000000000000000000000ED
:10A3700000000000000000000000000000000000DD
:10A3800000000000000000000000000000000000CD
:10A3900000000000000000000000000000000000BD
:10A3A00000000000000000000000000000000000AD
:10A3B000000000000000000000000000000000009D
:10A3C000000000000000000000000000000000008D
:10A3D000000000000000000000000000000000007D
:10A3E000000000000000000000000000000000006D
:10A3F000000000000000000000000000000000005D
:10A40000000000000000000000000000000000004C
:10A41000000000000000000000000000000000003C
:10A42000000000000000000000000000000000002C
:10A43000000000000000000000000000000000001C
:10A44000000000000000000000000000000000000C
:10A4500000000000000000000000000000000000FC
:10A46000FE55000000000000000000000000000099
:10A4700000000000000000000000000000000000DC
:10A480000005010202080308040805080608070879
:10A49000080609070A080B020C020D030E040F60E0
:10A4A00000000000000000000000000000000000AC
:10A4B000000000000000000000000000000000009C
:10A4C000000000000000000000000000000000008C
:10A4D000000000000000000000000000000000007C
:10A4E000000000000000000000000000000000006C
:10A4F000000000000000000000000000000000005C
:10A50000000000000000000000000000000000004B
:10A51000000000000000000000000000000000003B
:10A52000000000000000000000000000000000002B
:10A53000000000000000000000000000000000001B
:10A54000000000000000000000000000000000000B
:10A5500000000000000000000000000000000000FB
:10A5600000000000000000000000000000000000EB
:10A5700000000000000000000000000000000000DB
:10A5800000000000000000000000000000000000CB
:10A5900000000000000000000000000000000000BB
:10A5A00000000000000000000000000000000000AB
:10A5B000000000000000000000000000000000009B
:10A5C000000000000000000000000000000000008B
:10A5D000000000000000000000000000000000007B
:10A5E000000000000000000000000000000000006B
:10A5F000000000000000000000000000000000005B
:10A60000000000000000000000000000000000004A
:10A61000000000000000000000000000000000003A
:10A62000000000000000000000000000000000002A
:10A63000000000000000000000000000000000001A
:10A64000000000000000000000000000000000000A
:10A6500000000000000000000000000000000000FA
:10A6600000000000000000000000000000000000EA
:10A6700000000000000000000000000000001000CA
:10A6800000000000000000000000000000000000CA
:10A6900000000000000000000000000000000000BA
:10A6A00003B603E803B603E803B603E803B603E81A
:10A6B000000000000000000000000000000000009A
:10A6C0001E020E040E040E040E042802280240404E
:10A6D00040404040858585000000000400000004E3
:10A6E0000000040004040000000000020302000057
:10A6F0000000000103010000000000000000000055
:10A700000000000000000000000000000000000049
:10A710000000000000000000000000000000000039
:10A720000000000000000000000000000000000029
:10A730000000000000000000000000000000000019
:10A740000000000000000000000000000000000009
:10A7500000000000000000000000000000000000F9
:10A7600000000000000000000000000000000000E9
:10A7700000000000000000000000000000000000D9
:10A7800000000000000000000000000000000000C9
:10A7900000000000000000000000000000000000B9
:10A7A00000000000000000000000000000000000A9
:10A7B0000000000000000000000000000000000099
:10A7C0000000000000000000000000000000000089
:10A7D0000000000000000000000000000000000079
:10A7E0000000000000000000000000000000000069
:10A7F00044543137363742415243454C4F4E414520
:10A80000FF07F2168BFE48BD59C4FD11E4009DFC04
:10A810005EAB4FD2FB8D789C01FAC237D34EF99BC9
:10A820006E8A17F8D421C558F72ADF3BA6F6659043
:10A8300074E9F53CC92DB0F4738662FFF3A055B1FD
:10A840002CF2EF1AFE63F1B643A73AF0F90CE87563
:10A85000FFFFFFFFFFFFFFFFFFFFFFFFFFFFFFFF08
:10A86000FFFFFFFFFFFFFFFFFFFFFFFFFFFFFFFFF8
:10A87000FFFFFFFFFFFFFFFFFFFFFFFFFFFFFFFFE8
:10A88000FFFFFFFFFFFFFFFFFFFFFFFFFFFFFFFFD8
:10A89000FFFFFFFFFFFFFFFFFFFFFFFFFFFFFFFFC8
:10A8A000FFFFFFFFFFFFFFFFFFFFFFFFFFFFFFFFB8
:10A8B000FFFFFFFFFFFFFFFFFFFFFFFFFFFFFFFFA8
:10A8C000FFFFFFFFFFFFFFFFFFFFFFFFFFFFFFFF98
:10A8D000FFFFFFFFFFFFFFFFFFFFFFFFFFFFFFFF88
:10A8E000FFFFFFFFFFFFFFFFFFFFFFFFFFFFFFFF78
:10A8F000FFFFFFFFFFFFFFFFFFFFFFFFFFFFFFFF68
:10A90000FFFFFFFFFFFFFFFFFFFFFFFFFFFFFFFF57
:10A91000FFFFFFFFFFFFFFFFFFFFFFFFFFFFFFFF47
:10A92000FFFFFFFFFFFFFFFFFFFFFFFFFFFFFFFF37
:10A93000FFFFFFFFFFFFFFFFFFFFFFFFFFFFFFFF27
:10A94000FDF4EFFFFFFFFFFFFFFFFFFFFFFFFFFF34
:10A95000FFFFFFFFFFFFFFFFFFFFFFFFFFFFFFFF07
:10A96000FFFD00000000FBFE000000FFFDFF00FFF8
:10A97000FFFFF9FD0000FFFFFFFD00000000FFFFEB
:10A9800000000000FFFE00000000FCFD00000000D1
:10A99000FCFF00000000FCFE00000000FBFD0000CA
:10A9A0000000FBFF00000000FBFE00000000FBFDBC
:10A9B000000000FFFBFF000000FFFBFE000000FFA7
:10A9C000FEFD00000000FEFF00000000FEFE000093
:10A9D0000000FEFD000000FFFEFF000000FFFEFE85
:10A9E000000000FFFAFD00FFFFFFFAFF00FFFFFF7E
:10A9F000FAFE00FFFFFFFAFD0000FFFFFAFF000074
:10AA0000FFFFFAFE0000FFFFFAFD000000FFFAFF63
:10AA1000000000FFFAFE000000FFFAFD000000FF4A
:10AA2000FAFF000000FFFAFE000000FFFDFF00FF3C
:10AA3000FFFFFDFF00FFFFFFFDFE00FFFFFFFDFF2B
:10AA40000000FFFFFDFD0000FFFFFDFE0000FFFF17
:10AA5000FDFF000000FFFDFD000000FFFDFE000007
:10AA600000FFFDFF0000FFFFFDFD0000FFFFFDFEFA
:10AA70000000FFFFF9FF00000000F9FD00000000EA
:10AA8000F9FD00000000FFFF00000000FFFF0000D4
:10AA90000000FFFF00000000FFFF00000000FFFFBC
:10AAA00000000000FFFF00000000FFFF00000000AA
:10AAB000FFFF00000000FFFF00000000FFFF00009C
:10AAC0000000FFFF00000000FFFF00000000FFFF8C
:10AAD00000000000FFFF00000000FFFF000000007A
:10AAE000FFFF00000000FFFF00000000FFFF00006C
:10AAF0000000FFFF00000000FFFF00000000FFFF5C
:10AB000000000000FFFF00000000FFFF0000000049
:10AB1000FFFF00000000FFFF00000000FFFF00003B
:10AB20000000FFFF00000000FFFF00000000FFFF2B
:10AB300000000000FFFF00000000FFFF0000000019
:10AB4000FFFF00000000FFFF00000000FFFF00000B
:10AB50000000FFFF00000000FFFF00000000FFFFFB
:10AB6000FFFFFFFFFFFFFFFFFFFFFFFFFFFFFFFFF5
:10AB7000FFFFFFFFFFFFFFFFFFFFFFFFFFFFFFFFE5
:10AB8000FFFFFFFFFFFFFFFFFFFFFFFFFFFFFFFFD5
:10AB9000FFFFFFFFFFFFFFFFFFFFFFFFFFFFFFFFC5
:10ABA000FFFFFFFFFFFFFFFFFFFFFFFFFFFFFFFFB5
:10ABB000FFFFFFFFFFFFFFFFFFFFFFFFFFFFFFFFA5
:10ABC000FFFFFFFFFFFFFFFFFFFFFFFFFFFFFFFF95
:10ABD000FFFFFFFFFFFFFFFFFFFFFFFFFFFFFFFF85
:10ABE000FFFFFFFFFFFFFFFFFFFFFFFFFFFFFFFF75
:10ABF000FFFFFFFFFFFFFFFFFFFFFFFFFFFFFFFF65
:10AC0000FFFFFFFFFFFFFFFFFFFFFFFFFFFFFFFF54
:10AC1000FFFFFFFFFFFFFFFFFFFFFFFFFFFFFFFF44
:10AC2000FFFFFFFFFFFFFFFFFFFFFFFFFFFFFFFF34
:10AC3000FFFFFFFFFFFFFFFFFFFFFFFFFFFFFFFF24
:10AC4000FFFFFFFFFFFFFFFFFFFFFFFFFFFFFFFF14
:10AC5000FFFFFFFFFFFFFFFFFFFFFFFFFFFFFFFF04
:10AC600001AAFFFFFFFFFFFFFFFFFFFFFFFFFFFF47
:10AC7000FFFFFFFFFFFFFFFFFFFFFFFFFFFFFFFFE4
:10AC8000FFFAFEFDFDF7FCF7FBF7FAF7F9F7F8F727
:10AC9000F7F9F6F8F5F7F4FDF3FDF2FCF1FBF09FA0
:10ACA000FFFFFFFFFFFFFFFFFFFFFFFFFFFFFFFFB4
:10ACB000FFFFFFFFFFFFFFFFFFFFFFFFFFFFFFFFA4
:10ACC000FFFFFFFFFFFFFFFFFFFFFFFFFFFFFFFF94
:10ACD000FFFFFFFFFFFFFFFFFFFFFFFFFFFFFFFF84
:10ACE000FFFFFFFFFFFFFFFFFFFFFFFFFFFFFFFF74
:10ACF000FFFFFFFFFFFFFFFFFFFFFFFFFFFFFFFF64
:10AD0000FFFFFFFFFFFFFFFFFFFFFFFFFFFFFFFF53
:10AD1000FFFFFFFFFFFFFFFFFFFFFFFFFFFFFFFF43
:10AD2000FFFFFFFFFFFFFFFFFFFFFFFFFFFFFFFF33
:10AD3000FFFFFFFFFFFFFFFFFFFFFFFFFFFFFFFF23
:10AD4000FFFFFFFFFFFFFFFFFFFFFFFFFFFFFFFF13
:10AD5000FFFFFFFFFFFFFFFFFFFFFFFFFFFFFFFF03
:10AD6000FFFFFFFFFFFFFFFFFFFFFFFFFFFFFFFFF3
:10AD7000FFFFFFFFFFFFFFFFFFFFFFFFFFFFFFFFE3
:10AD8000FFFFFFFFFFFFFFFFFFFFFFFFFFFFFFFFD3
:10AD9000FFFFFFFFFFFFFFFFFFFFFFFFFFFFFFFFC3
:10ADA000FFFFFFFFFFFFFFFFFFFFFFFFFFFFFFFFB3
:10ADB000FFFFFFFFFFFFFFFFFFFFFFFFFFFFFFFFA3
:10ADC000FFFFFFFFFFFFFFFFFFFFFFFFFFFFFFFF93
:10ADD000FFFFFFFFFFFFFFFFFFFFFFFFFFFFFFFF83
:10ADE000FFFFFFFFFFFFFFFFFFFFFFFFFFFFFFFF73
:10ADF000FFFFFFFFFFFFFFFFFFFFFFFFFFFFFFFF63
:10AE0000FFFFFFFFFFFFFFFFFFFFFFFFFFFFFFFF52
:10AE1000FFFFFFFFFFFFFFFFFFFFFFFFFFFFFFFF42
:10AE2000FFFFFFFFFFFFFFFFFFFFFFFFFFFFFFFF32
:10AE3000FFFFFFFFFFFFFFFFFFFFFFFFFFFFFFFF22
:10AE4000FFFFFFFFFFFFFFFFFFFFFFFFFFFFFFFF12
:10AE5000FFFFFFFFFFFFFFFFFFFFFFFFFFFFFFFF02
:10AE6000FFFFFFFFFFFFFFFFFFFFFFFFFFFFFFFFF2
:10AE7000FFFFFFFFFFFFFFFFFFFFFFFFFFFFEFFFF2
:10AE8000FFFFFFFFFFFFFFFFFFFFFFFFFFFFFFFFD2
:10AE9000FFFFFFFFFFFFFFFFFFFFFFFFFFFFFFFFC2
:10AEA000FC49FC17FC49FC17FC49FC17FC49FC1742
:10AEB000FFFFFFFFFFFFFFFFFFFFFFFFFFFFFFFFA2
:10AEC000E1FDF1FBF1FBF1FBF1FBD7FDD7FDBFBFCE
:10AED000BFBFBFBF7A7A7AFFFFFFFFFBFFFFFFFB19
:10AEE000FFFFFBFFFBFBFFFFFFFFFFFDFCFDFFFF85
:10AEF000FFFFFFFEFCFEFFFFFFFFFFFFFFFFFFFF67
:10AF0000FFFFFFFFFFFFFFFFFFFFFFFFFFFFFFFF51
:10AF1000FFFFFFFFFFFFFFFFFFFFFFFFFFFFFFFF41
:10AF2000FFFFFFFFFFFFFFFFFFFFFFFFFFFFFFFF31
:10AF3000FFFFFFFFFFFFFFFFFFFFFFFFFFFFFFFF21
:10AF4000FFFFFFFFFFFFFFFFFFFFFFFFFFFFFFFF11
:10AF5000FFFFFFFFFFFFFFFFFFFFFFFFFFFFFFFF01
:10AF6000FFFFFFFFFFFFFFFFFFFFFFFFFFFFFFFFF1
:10AF7000FFFFFFFFFFFFFFFFFFFFFFFFFFFFFFFFE1
:10AF8000FFFFFFFFFFFFFFFFFFFFFFFFFFFFFFFFD1
:10AF9000FFFFFFFFFFFFFFFFFFFFFFFFFFFFFFFFC1
:10AFA000FFFFFFFFFFFFFFFFFFFFFFFFFFFFFFFFB1
:10AFB000FFFFFFFFFFFFFFFFFFFFFFFFFFFFFFFFA1
:10AFC000FFFFFFFFFFFFFFFFFFFFFFFFFFFFFFFF91
:10AFD000FFFFFFFFFFFFFFFFFFFFFFFFFFFFFFFF81
:10AFE000FFFFFFFFFFFFFFFFFFFFFFFFFFFFFFFF71
:10AFF000BBABCEC8C9C8BDBEADBCBAB3B0B1BEBA9A
:00000001FF
